:100000000C94AA000C9420020C94C7000C94C70016
:100010000C94C7000C94C7000C94C7000C94C70044
:100020000C94C7000C94C7000C94C7000C94C70034
:100030000C94C7000C94C7000C94C7000C94C70024
:100040000C94C7000C94C7000C94C7000C94C70014
:100050000C94C7000C94C7000C94C7000C94C70004
:100060000C94C7000C94C700180372006100700064
:1000700068006E00650074002E006E00650074005C
:10008000040309040A033100300030003000050188
:100090000904A1010901A1008501093009311500F8
:1000A00026FF007508950281020509190129081526
:1000B000002501750195088102C0C005010904A150
:1000C000010901A100850209300931150026FF0050
:1000D00075089502810205091901290815002501F5
:1000E000750195088102C0C005010904A10109013B
:1000F000A100850309300931150026FF0075089518
:1001000002810205091901290815002501750195CB
:10011000088102C0C005010904A1010901A10085EF
:100120000409300931150026FF0075089502810287
:100130000509190129081500250175019508810295
:10014000C0C012010101000000089B280300050146
:100150000102030111241FBECFEFD4E0DEBFCDBFEB
:1001600011E0A0E0B1E0E0EBFEE002C005900D92EE
:10017000A635B107D9F721E0A6E5B1E001C01D928F
:10018000A53BB207E1F70E9477060C9456070C9442
:100190000000CF93C62F2091000124FF0BC02091B7
:1001A0008B0138E8232720938B01FC01ACE8B1E0F8
:1001B0008C2F04C02AE520930001F7CF815018F05E
:1001C00091919D93FBCF6C2F8CE891E00E941C02D3
:1001D000CC5FC0930001CF910895CF93DF938091BE
:1001E0009B0118160CF0AEC09091980120919701D8
:1001F0002D3219F090E880E09FC02AE5209301019C
:100200008B30C1F7CCE0D0E0C91BD109C156DE4F1D
:100210008881807609F080C01092890189818111DE
:100220000BC010928A0189E891E090939A01809323
:10023000990190E882E079C0853021F48A81809329
:100240009C0171C0863009F04BC08B81813009F46C
:1002500042C0823021F4CE010E94830360C083300B
:1002600069F58A81811109C080E890E090939A0134
:100270008093990190EC84E058C0813049F488E67D
:1002800090E090939A018093990190EC88E14DC0A1
:10029000823049F485E291E090939A01809399012C
:1002A00090E880E242C08330E1F584E890E09093EA
:1002B0009A018093990190EC8CE037C0813249F427
:1002C00089E691E090939A018093990190EC89E0FE
:1002D0002CC0823231F5CE010E94830390EC25C000
:1002E000883019F48EE991E00AC0893021F48A81BE
:1002F00080939E0118C08A3049F489E891E0909378
:100300009A018093990190E881E00FC08B3059F4F5
:1003100083EC80938B0107C0CE010E94B10390E86B
:1003200004C090EC01C090E880E02F81211104C04E
:100330002E81281708F4822F909356018093020192
:1003400010929B018091010184FF46C080910201BF
:100350008F3F09F441C0C82F893008F0C8E08C1BDA
:10036000809302012091560120FD02C0DBE401C010
:10037000D3EC2F5F209356018091990190919A01BF
:1003800026FD05C0FC01A1E8B1E02C2F0AC0A1E8C0
:10039000B1E0FC012C2F215048F034913D9331966F
:1003A000FACF215018F031913D93FBCF8C0F911D66
:1003B00090939A01809399016C2F81E891E00E94BB
:1003C0001C0284E08C0FC83019F09FEF909302015B
:1003D000D0938001809301018AE099B1957031F446
:1003E0008150D9F710929C0110929601DF91CF9124
:1003F0000895E9E6F0E0808183608083E89A83ECE9
:1004000080938B010895A82FB92F8FEF9FEF41E0C4
:1004100050EA615070F02D9138E0722F7827969550
:100420008795269570FF02C0842795273A95A9F7EE
:10043000F0CF809590950895E6DF8D939D93089574
:10044000CF93CFB7CF93489BFECF489B09C0489B23
:1004500007C0489B05C0489B03C0489B01C09EC085
:10046000DF93C0919801DD27C156DE4F489B02C043
:10047000DF91EBCF2F930F931F9309B12FEF00FB69
:1004800020F94F933F9319B14FEF012700FB21F95A
:100490003BE031C04E7F012F19B1216028C0102FE1
:1004A0004D7F2260000009B129C04B7F2460012FDD
:1004B000000019B12BC019B1477F28602AC04F7EB8
:1004C00009B120612CC04F7D19B120622FC04F7B34
:1004D00009B1206432C0422709B149934FEF0000AF
:1004E000102710FB20F919B11570A9F1297F91F29D
:1004F000012700FB21F909B1237F89F23150F0F186
:10050000102710FB22F919B1277E79F2012700FB91
:1005100023F92F7C81F209B1102710FB24F92F79E0
:1005200071F200C019B1012700FB25F92F7359F2B0
:1005300000C009B1102710FB26F9223040F200C09C
:1005400019B1012700FB27F9243028F64F772068DE
:1005500019B10000F9CF3B503195333011E01CBB8D
:10056000B8F0C31BD0400881033C41F10B3431F19A
:100570001981412F1F7720919601121731F4093606
:1005800091F10D3279F0013E69F0222720939D010F
:100590003F914F911F910F912F91DF91CF91CFBF3D
:1005A000CF91189500939D013F914F911F910F910D
:1005B0002F91DF91CCB3C0FD46CFF0CF00919D01CC
:1005C000002331F310919B011123A1F53430A2F1E6
:1005D00030939B0100939701109198013BE0311BF0
:1005E0003093980129C000919B0101301CF50AE568
:1005F00047FD09C03091010134FD20C00093010185
:10060000C0E8D1E01FC03091000134FD17C0009355
:100610000001CBE8D1E016C0052710E00BB91FC0E0
:10062000052722C0052727C005272CC0052710E075
:100630000BB933C04AE503C042ED01C0432FC4E10A
:10064000D0E032E01AB11560589A0BB11AB95F9335
:1006500055E020E820FF05270BB9279517951C3F8B
:10066000D8F620FF052727950BB917951C3FC0F634
:1006700020FF0527279517950BB91C3F98F620FFFB
:100680000527279517951C3F0BB970F600C04991B7
:1006900020FF05270BB9279517951C3F38F620FF3B
:1006A000052727950BB917951C3F38F520FF05271F
:1006B000279517950BB91C3F10F520FF05272795A7
:1006C00017951C3F0BB9E8F4242F3A9519F60A7FC9
:1006D0005F910BB900C010919C01C651D04011F040
:1006E0001093960111E01CBB01601AB11A7F402FD4
:1006F0004A7F0BB91AB94BB94BCF0527D3CF052782
:10070000D8CF0527DDCFFC018081807641F591812E
:10071000963031F593819230D1F0923269F0913078
:10072000F9F4809168019091690190939A01809306
:10073000990180916701089580916B0190916C01FE
:1007400090939A018093990180916A01089583E0C2
:1007500091E090939A018093990182E2089580E05C
:100760000895DC0189E591E090939A0180939901C5
:100770008C918076803299F411968C91119781300A
:1007800071F410925801E0916501F09166010784BF
:10079000F089E02D12966C9189E591E0099480E052
:1007A000089586FB992790F9482F407850E023E080
:1007B000559547952A95E1F7942B482F407250E0C4
:1007C00033E0559547953A95E1F7942B8071282FA2
:1007D00030E035952795892F822B089581502091FF
:1007E0006E0190E0222369F0DC01A858BE4FFC01A5
:1007F000E059FE4F81E02C91908129130DC080E0DB
:100800000895880F991FBC0160597E4F42E050E067
:1008100088589E4F0E944907089580916E01882351
:1008200009F445C0449A20E32A95F1F7449888E0FA
:1008300090E040E050E068E16A95F1F74598550F87
:10084000440F339B5160329B416028E12A95F1F7B8
:10085000459A0197009779F788E090E020E030E032
:1008600068E16A95F1F74598330F220F339B3160A9
:10087000329B216068E16A95F1F7459A01970097EC
:1008800079F788E090E068E16A95F1F7459868E1CA
:100890006A95F1F7459A01970097A9F75093780167
:1008A0004093790130937A0120937B0108958091E0
:1008B0006D01449A882309F468C080E38A95F1F7B2
:1008C000449820E32A95F1F72D9A68E16A95F1F7AB
:1008D00088E090E040E050E0459828E12A95F1F763
:1008E000550F440F339B5160329B4160459A68E13C
:1008F0006A95F1F70197009779F750937801409343
:100900007A0188E090E0459828E12A95F1F756951C
:100910004695339B5068329B4068459A68E16A95DA
:10092000F1F70197009779F72D9888E18A95F1F70B
:1009300088E090E020E030E0459868E16A95F1F7C2
:10094000330F220F339B3160329B2160459A68E15F
:100950006A95F1F70197009779F730937C0120931E
:100960007E0188E090E0459868E16A95F1F7369558
:100970002695339B3068329B2068459A68E16A95DA
:10098000F1F70197009779F742C080E38A95F1F774
:10099000449888E090E020E030E040E050E068E1FA
:1009A0006A95F1F74598550F440F330F220F339B8B
:1009B0005160329B4160319B3160309B216068E126
:1009C0006A95F1F7459A0197009749F75093780196
:1009D00040937A0130937C0120937E0188E090E07F
:1009E00068E16A95F1F745985695469536952695AE
:1009F000339B5068329B4068319B3068309B206845
:100A000068E16A95F1F7459A0197009749F7809157
:100A10005401882321F180916F015F3F11F48160BF
:100A200001C08E7F80936F0180916F014F3F11F461
:100A3000826001C08D7F80936F0180916F013F3F85
:100A400011F4846001C08B7F80936F0180916F01EE
:100A50002F3F11F4886001C0877F80936F018091E0
:100A60006F0180FD50E05093790181FD40E040939B
:100A70007B0182FD30E030937D0183FD20E02093F7
:100A80007F010895CF93CFB7F8943C9A3D9A87B1F0
:100A9000807F87B988B18F6088B9459A4498259A34
:100AA0002D9A10926F010E940D04809154018111C2
:100AB00024C0809179018F3F29F480916F0181607A
:100AC00080936F0180917B018F3F29F480916F01AA
:100AD000826080936F0180917D018F3F29F4809126
:100AE0006F01846080936F0180917F018F3F29F4B3
:100AF00080916F01886080936F01449A40E34A952A
:100B0000F1F7449830E020E080E090E048E14A9539
:100B1000F1F74598339905C08331910519F431E017
:100B200001C02F5F48E14A95F1F7459A0196883157
:100B3000910561F7332329F0273119F481E080937F
:100B40006E012D98329B0FC0449A80E38A95F1F78D
:100B5000329909C0449840E34A95F1F7329B03C0AB
:100B600081E080936D012D9A329B0FC0449A80E3FF
:100B70008A95F1F7329909C0449840E34A95F1F714
:100B8000329B03C081E080936D01CFBFCF91089568
:100B9000EF92FF920F931F93CF93DF93EC01653099
:100BA00008F08EC080916E01E62EFF24E7FCF094E1
:100BB000882349F181E0E81AF108870108581E4F9F
:100BC0002097D1F06883D8019C9190FD02C080E805
:100BD00001C08FEF91FD80E08983F801908192FD43
:100BE00002C080E801C08FEF93FD80E08A83D801C6
:100BF0008C910E94D1038B83F701E059FE4FD801FD
:100C00008C9180835BC0B1E0EB1AF1088701000F83
:100C1000111F209709F448C06883F801E858FE4F77
:100C2000908190FD02C080E801C08FEF91FD80E0CF
:100C30008983908192FD02C080E801C08FEF93FD0F
:100C400080E08A8380916F0190E002C0959587953E
:100C5000EA94E2F780FF05C080810E94D1038B8374
:100C600023C08081482F441F4427441F2181E0E195
:100C70002E9F90011124422B282F207430E065E034
:100C8000359527956A95E1F7422B282F207230E0A1
:100C900073E0359527957A95E1F7422B807190E0C6
:100CA00095958795482B4B83F801E059FE4FD80165
:100CB000A858BE4F8D919C919183808384E001C0A0
:100CC00080E0DF91CF911F910F91FF90EF900895F9
:100CD0001092540108958EE890E09093470180931C
:100CE000460183E491E0089582E190E0089581E077
:100CF00084B98EEF85B917B88FEF88B988EF8BB9B3
:100D000085E08AB982E08093B00087E08093B100EB
:100D100084EC8093B3008FE295E70197F1F700C070
:100D2000000083B18670843011F40E9468060E942E
:100D30006B06FC0190936601809365018381948129
:100D400090936C0180936B01818180936A0187810C
:100D50009085009731F090936901809368018581B7
:100D600008C082E491E090936901809368010E9439
:100D700074068093670180916A0180931C018BB196
:100D80008A7F8BB98AB185608AB987EC9FEA01971F
:100D9000F1F700C000008AB18A7F8AB9E09165014D
:100DA000F09166010184F285E02D09950E94F90118
:100DB000E0916501F09166010384F485E02D0995C9
:100DC000789482E0D82E01E010E0A8950E94ED0012
:100DD000B99BFBCFD7BAE0916501F091660103841E
:100DE000F485E02D0995C0E0D0E0E12CE0916501AB
:100DF000F09166018081992787FD9095C817D907E2
:100E00008CF40584F685E02D8C2F8F5F099588235F
:100E100039F0C8010C2E01C0880F0A94EAF7E82ABD
:100E20002196E4CFEE2089F2C0E0D0E0FF24E7FC79
:100E3000F094E0916501F09166018081992787FD2A
:100E40009095C817D9070CF0C0CFC7010C2E02C06F
:100E5000959587950A94E2F780FF19C0809100016B
:100E600084FF15C00784F089E02D6C2F6F5F89E542
:100E700091E00995682F89E591E00E94C900809171
:100E8000000184FD04C00E94ED00A895F8CF2196D2
:100E9000D0CFFB01DC0104C08D910190801921F4B9
:100EA00041505040C8F7881B990B0895F894FFCF24
:100EB0005A5AFF0902220001010080320904000091
:100EC00001030000000921010100012200000705C3
:100ED000810308000A1E0334006E006500730034AD
:100EE0000073006E00650073002000760031002E54
:100EF00000350004B40000000000000042050D04AD
:060F0000EE03C80501002C
:00000001FF
